:020000041001E9
:200000000088000841E620101D36011021360110000000000000000000000000000000002D
:200020000000000000000000000000003D36011000000000000000003F360110413601102E
:20004000433601104536011047360110F1370110493601104B3601104D3601104F36011077
:2000600051360110533601105536011057360110593601105B3601105D3601105F36011088
:020000041020CA
:20E6400072B6002000210022002300240025002600270B4880F308880A480B490860BFF360
:20E660004F8F05F624F8094FB847094A094C00231360121DA242FBD302F60FFBFEE700BF89
:20E68000008800080000011008ED00E06136011000480008D860000800480008FF870008EE
:020000041001E9
:2006400000002110422063308440A550C660E770088129914AA16BB18CC1ADD1CEE1EFF19A
:200660003112100273325222B5529442F772D662399318837BB35AA3BDD39CC3FFF3DEE35A
:200680006224433420040114E664C774A44485546AA54BB528850995EEE5CFF5ACC58DD51A
:2006A0005336722611163006D776F6669556B4465BB77AA719973887DFF7FEE79DD7BCC7DA
:2006C000C448E5588668A7784008611802282338CCC9EDD98EE9AFF9488969990AA92BB99A
:2006E000F55AD44AB77A966A711A500A333A122AFDDBDCCBBFFB9EEB799B588B3BBB1AAB5A
:20070000A66C877CE44CC55C222C033C600C411CAEED8FFDECCDCDDD2AAD0BBD688D499D19
:20072000977EB66ED55EF44E133E322E511E700E9FFFBEEFDDDFFCCF1BBF3AAF599F788FD9
:200740008891A981CAB1EBA10CD12DC14EF16FE18010A100C230E320045025404670676099
:20076000B9839893FBA3DAB33DC31CD37FE35EF3B1029012F322D232354214527762567259
:20078000EAB5CBA5A89589856EF54FE52CD50DC5E234C324A0148104667447642454054419
:2007A000DBA7FAB79987B8975FE77EF71DC73CD7D326F2369106B0165766767615463456D9
:2007C0004CD96DC90EF92FE9C899E9898AB9ABA94458654806782768C018E1088238A32899
:2007E0007DCB5CDB3FEB1EFBF98BD89BBBAB9ABB754A545A376A167AF10AD01AB32A923A59
:200800002EFD0FED6CDD4DCDAABD8BADE89DC98D267C076C645C454CA23C832CE01CC10C18
:200820001FEF3EFF5DCF7CDF9BAFBABFD98FF89F176E367E554E745E932EB23ED10EF01ED8
:2008400000050000F510011001050000490E011002050000551101100305000099110110CE
:2008600004050000AD120110050400007D1201100605000025110110951701101900881333
:20088000010201009D1701101900881301020200D1160110000000000000000010010200CB
:2008A00025160110000000000000000011010200551F011061200110AD20011022010200BE
:2008C00099250110000000000000000027020000D5200110492201105F2201103101020CCC
:2008E0006D2A0110000000000000000034020000F12601106B2801101329011036020001C8
:200900005D290110E12901103D2A0110370200033518011000000000000000003E010200D2
:2009200001000000C51601100000000000D101000000000021D001000007031011F11800D2
:200940001807031013F11800380703108CF11000A80703100EF11800C807031062F101005B
:20096000F807031088F118001808031024F118006807031022F118004807031071F11800EB
:20098000000000005BD0010000000000C5EE02000000000094EE0A0071220110BB22011058
:2009A00000FF0C000100007101FF0048720000009B240110E9240110040304000100007195
:2009C0000103044A100000003D2301106123011001FF0C000100007101FF014A10000000D6
:2009E00040420F0040420F0040420F0040420F0006070000E0070000DF070000E8070000EA
:200A000000000000790E0110B30E0110C5180110F51901102F190110DB190110351A0110A1
:200A2000451A0110551A01104D1A0110D51B0110F51D0110851101108D110110C9110110E9
:200A4000D7110110351201103D310110312C0110953101109F3101100912011089320110A8
:200A60009532011001330110DD120110EB120110F3120110FB12011011130110CF130110EF
:200A8000F71301103314011000000040000400000103060507090000010706020308050A56
:200AA0000102030A0F000000010A0B0C070D0E000A0703000601070308050000000102039B
:200AC000040506000000000014360110245C0008B40400000600000000010203040506074A
:200AE000080C101418203040080C101418203040000102030405060708090909090A0A0AD0
:200B00000A0B0B0B0B0C0C0C0C0D0D0D0D0D0D0D0D0E0E0E0E0E0E0E0E0E0E0E0E0E0E0E35
:200B20000E0F0F0F0F0F0F0F0F0F0F0F0F0F0F0F0F0000005C0B0110B05B0008B00B011060
:200B4000B80B0110D05B00080000000000000000C80B01100102020101000100CC0B0110BA
:200B600000000000CC0B0110010078080800000000000001000053400080000001000000EF
:200B80000000524002077808E00B01100007080000000000020000077808000000000000A6
:200BA0000000010780080000010000000000000000000000000101000000000000000000A2
:200BC0000100000000FF0000000000001000F4010207020002070201FF00D007040000001F
:200BE000E0070000DF07000000000000000000000000000000000000000000000000000028
:200C0000000000000000000000043140010000000000000008000000150000000000000041
:200C20000000000000000000000000000000000000000000000000000000000000000000B4
:200C4000000000000004314000000000010000000E000000150000000000000000000000FB
:200C6000000000000000000000000000000000000000000000000000000000000000000074
:200C80000400000000000000000000000000000000000000704772B6704700B500F002F81B
:200CA000002000BD00B502F0C9FD00F00FF80121062000F031F80121084600F02DF80121EB
:200CC000002000F029F800F007F800BD0149002008707047AE58000870B581B000F0F2F860
:200CE00000F0F9FE00F07EFA534908780028F5D0524908780728F1D282008118504A490091
:200D00008A185049C0000818537A4468107AC11AC9B29818A047E1E770B507284CD283000B
:200D2000C218474B52009B181C7A082C0ED2002203E09D5C8D4202D00132A242F9D3D2B292
:200D4000A24203D19954197A013119723A4C3B492278002A07D12278072A2DD222788854B8
:200D60000120207028E0374DC200AA185678002217E08B5C834217D0DB00EB185B78B34292
:200D80000DD2237803E04D1EED5CCD54013B9342F9D8DBB2C85423780133237004E001321D
:200DA000D2B223789A42E4D323789A4204D12278885420780130207070BD10B5072839D23A
:200DC0008300C2181E4B52009B185A7A13E09C5C8C420ED100219954597A8A420ED101311E
:200DE00059721A7AC9B2914208D100215972197204E00132D2B21C7AA242E8D31A7A002A68
:200E000018D10D4913E00D4B9C5CA0420DD104E0D018407898540132D2B2087801388242EC
:200E2000F6D308780138087004E00132D2B20B789A42E8D310BD00BFAE580008B058000859
:200E4000B858000840080110F0B505460E4600240DE02F5D39460120FFF7AFFF7A1ED2B2E0
:200E6000022A03D203489200105880470134B442EFD3F0BD040A011000B59949002008707D
:200E80009849087098490870984902015218013010731328F8D3C0B200014018FF21017339
:200EA000002002F011FD0021C943002002F040FD00BD00B58B490020087002F057FD02F080
:200EC00076FD00BDF0B586B0864F00220292387800286FD0864C104602F05EFD064620681C
:200EE0000021864200D2012105917D4926600025097801913978049159E0019A7B4910010C
:200F00004418217B0091D1B2E07A0391012808D10598012843D10020E072606886423ED3E8
:200F200005E06068864202D20598012837D1A17A607AFFF7F1FE207A012809D12068801902
:200F40006060B04201D9002000E00120E07226E0387863490138387008780199884204D196
:200F6000217B5F480091017014E00499481E85420298034606D15D4A00018018FF210173E0
:200F8000009107E0594A00018118207B08730090DAB203925449019A087820730A70039875
:200FA000C0B202900098C0B201900135EDB204988542A2D306B0F0BDF9B581B00F460293B9
:200FC0001146019004467D20C00004F07BFA8100401A49014018C60004D139462046FFF726
:200FE0009BFE41E000240136204602F0D5FC3C4A00902546117811E03C4C09010C19617A26
:201000000198884207D1A17A8F4204D101983946FFF7D3FE06E0217B0135EDB231480378AA
:201020009D42E9D3142D1FD22E4801788D420FD1013101702C482D4A01780C01A418227BD8
:201040000270274802782273017001986072A772029820720098266031186160814201D9BA
:20106000002100E00121E17201B0F9BDF0B581B01B4A00240094167826E01C4F3201D51980
:201080006A7A90421CD1AA7A914219D1FFF795FE1449087801380870002C03D11049287BB9
:2010A000087008E0C0B2FF21844200D0297B00980001C01901730C49087828730E7007E049
:2010C00000962E7B0134E4B2064B1A789442D4D301B0F0BD00B5002002F05EFC00BD00BFAB
:2010E00002590008015900080059000804590008385B0008F0B505460E4600240DE02F5DE9
:2011000039460020FFF759FE7A1ED2B2042A03D203489200105880470134B442EFD3F0BD1E
:201120000C0A0110F0B505460E4600240DE02F5D39460620FFF741FE7A1ED2B2052A03D2AD
:2011400003489200105880470134B442EFD3F0BD1C0A0110F0B505460E4600240DE02F5DD1
:2011600039460220FFF729FE7A1ED2B2032A03D203489200105880470134B442EFD3F0BDED
:20118000300A011000B500F042FE00BD00B5002000F046FE00BD0000F0B505460E46002434
:2011A0000DE02F5D39460320FFF707FE7A1ED2B2082A03D203489200105880470134B442BF
:2011C000EFD3F0BD3C0A011000B500F015F809490120087000BD00B500F012F805490020D2
:2011E000087000BD00B503490878012801D100F04EFE00BD445A000800B502F03DF800BD06
:2012000000B502F03DF800BD00B501F0B5FE00BD60B581B0084E3578012D08D10093074DE8
:2012200013460A460146287801F0B4FC00E0002001B060BD704700BF455A0008475A0008E9
:2012400000B50B4A10700B4A117005210420FFF763FD00BD064908707047074908707047D4
:2012600000B5104600F090F900BD014908787047455A0008475A0008465A0008F0B50546C4
:201280000E4600240DE02F5D39460520FFF795FD7A1ED2B2032A03D2034892001058804707
:2012A0000134B442EFD3F0BD5C0A0110F0B505460E4600240DE02F5D39460420FFF77DFD29
:2012C0007A1ED2B2082A03D203489200105880470134B442EFD3F0BD680A011000B56E4956
:2012E0000320087000F02AFE00BD00B500F027FE00BD00B500F07AF900BD00B5674908783D
:20130000012802D100F0CCFD01E000F0E3FD00BDF0B585B06A46002003AF019078803B1F6B
:20132000191F981DFFF774FF04907A88694649C90546002A11D05A4C5A4F21780801C019E0
:2013400082811F46E0C0049AC270012201318270C9B2052004F0D4F821700020514A0101C0
:201360008C18A17B01292CD14F490878012805D04E490878012801D100F034F8474DA168A5
:201380004B480A782B783E2A0DD1E27B002B01D1427000E0027023686268A08900F04AFA3F
:2013A0000020A07311E0002B0FD1E27B4270414862680260404823680360A08900F082F831
:2013C000EEE70130C0B20528C8D305B0F0BD00B53A4A012303210420FFF7EEFD3349012048
:2013E000087000BD00B503210420FFF73FFE2F4A0020107000BD00B528490878002817D0FD
:20140000254A2F491078000140184068804701280ED104210846FFF729FE204A002008214A
:2014200010700320FFF778FC05210420FFF774FC00BD30B504210846FFF718FE1649204C03
:20144000087800010019806880471B490B681949114D0A680146287800010019007B00F0CE
:201460006DF80E4D0020287030BD30B512480A4D03681048124C7821026828780001001993
:20148000007B00F05BF830BD034A0D49107800014018007B704700BF9A5A0008985A000836
:2014A0003C5B0008485A0008995A00089D5A00089B5A00081448000810480008404B4C0051
:2014C00090080110F1B581B001900D4616461F4600244D4A21018A182878117B88421FD182
:2014E000002101B48B1849485B7B0078834201BC08D001310229F4D33B4632467F2100F08D
:201500001DF811E042493B460C701068324600900198294601B40198844601BCE04703E0D6
:201520000134E4B2092CD4D3092C05D13B4632462878112100F002F801B0F1BD30B5354D7E
:201540000C462978344D002901D1697800E02978002909D1112C07D3122C14D9312C12D036
:201560007E2C01D37F2C0ED994707F2150701170032018800821FFF7CFFB782C03D0052135
:201580000420FFF7C9FB30BD00B5204A117801291CD0204A1178002901D0002816D11F495E
:2015A0000878002808D11E4A012303210420FFF703FD1A4901200870154A134910780001A0
:2015C0004018007B312801D100F0AEFF104A0E49107800014018007B112802D100F06AF805
:2015E00003E0102801D100F00DF900BD00B500F0E2F900BD05490870704706490870704713
:2016000002490878704700BF90080110995A00089A5A0008985A00089B5A00089D5A0008F3
:20162000404B4C00F0B516461F460D464978264B4C06640E00221A70511CC9B2012906D38D
:2016400003D003290FD314D001E0022813D30132052AF1D31D4A506880476878000614D5F9
:20166000FFF7C4FF16E0194B1978A142EFD0122102E00228EBD013213B4632461120FFF7D6
:201680005DFF11490120087004E03A463146204600F001F8F0BD00B5512348700B700220A6
:2016A000108008210320FFF737FB05210420FFF733FB00BD00B504490878002801D1FFF789
:2016C00095FF00BD704700BF9E5A000820090110F0B581B00C46497815464A06520E009283
:2016E0004E4A1E4600231370591CC9B2012906D303D0032923D337D001E0022836D3013311
:20170000052BF1D3464B474F18788100081A8000C0598047424B18788100081A8000C01902
:20172000414B807A1870617809062CD5012827D03E4A012303210420FFF73EFC28E0002145
:201740008F007A1A374F9200D219927A009FBA4202D1334A117002E001310229F0D3C9B26E
:201760000229CCD1122102E00228C8D0132133462A461020FFF7E2FE28490120087007E0B6
:20178000FFF734FF04E032460098294600F00DF801B0F0BD00B500F0A5FF00BD00B5244942
:2017A0000020087000F098FF00BD70B515460C4600218B005A1A1B4B9200D218937A8342A7
:2017C0001CD15021217060709088010AA170E070D68831460520400203F074FE207130461E
:2017E00003F068FE60710620288008210320FFF793FA05210420FFF78FFA02E0013102291A
:20180000D7D370BD00B505490878002805D106490878012801D1FFF7E9FE00BDA05A00080A
:201820009F5A000878080110995A0008404B4C00985A000870B54E7875066D0E0024611CC8
:20184000C9B2012906D303D003291AD31DD001E002281CD30134032CF1D330061CD515498A
:201860000878012825D014490878002821D1134A012303210420FFF79FFB11490120087087
:2018800017E0002DE6D0122102E00228E2D013213E20FFF753FE0CE07E20107055700220B3
:2018A000188008210320FFF737FA05210420FFF733FA70BD995A0008985A0008404B4C00B7
:2018C0009D5A000830B55449002008700120FFF791FE524C00202070022000F009FA05469B
:2018E0001020FFF7B7FC4E48854204D101202070FFF7B0FC01E0002020702078002810D059
:20190000FFF7ABFC01F06DFE00F031F8022000F0CFF9FFF7AAFC012808D10220FFF76AFEBD
:2019200004E00120FFF766FE00F001F830BD00B5FFF766FE012812D1032000F0D9F93849F1
:20194000364A884201D0002000E001201070002805D000F022F833490120087003E001F0DB
:2019600040FE00F004F830490120087000BD00B5FFF791F901210420FFF7CEF901210320F1
:20198000FFF7CAF901210220FFF7C6F900BD00B5264801210843804700BD00B502210120CB
:2019A000FFF7BAF902210846FFF7B6F902210020FFF7B2F900BD00B502210320FFF7ACF931
:2019C00002210120FFF7A8F902210846FFF7A4F902210020FFF7A0F900BD00B5114908780A
:2019E000012802D1FFF7D9FF03E0022801D1FFF7E2FF00BD00B50B490878012804D1002003
:201A00000870FFF7C4FF05E009490878012801D001F046FF00BD0000A35A0008A15A0008E9
:201A2000AA55AA5500480008A25A0008400604100148000800B5062002F005F8674901200E
:201A4000087000BD00B500F009F800BD00B500F01AF800BD00B500F00CF800BD00B5604AB5
:201A6000032010705F4A11685F4A106802F02EF800BD00B55B4B1A685B4B19685B4B186881
:201A800002F081F800BD70B557490D6855490C6856490E68FFF7F8FC55490870E00FC00707
:201AA00002D00120640064085249087052490878002806D151490D60514908604E49012075
:201AC0000870474B022018704C4B22463146186800F028F870BD00B540490878012805D162
:201AE00002F0C3F8022801D102F001F800BD70B5434B0446002018603F4B0D46164618703F
:201B0000FFF7C2FC3F493A4B611A1D2218701204914205D232462946204602F093F800E058
:201B2000002070BDF1B5384B0D4614461A7A0026002A01D1082C29D231461F46082A08D2B5
:201B4000A14214D2685CB85401321A72D2B20131F4E72E48621A4919026008241D462C48E3
:201B6000274A01601168091911601E7228E021480178012901D1114612E0194A1670254A70
:201B80001178254A1078FFF7C7F814E01F486107490F0160641A6119E1E7FF2078540131B7
:201BA0000829FAD31648012608240168891801601D460021197215480021012E016008D115
:201BC0000E4A00981168091911602246294601F069FFF1BD00B500F0BBF800BDAB5A000809
:201BE000AA5A000818480008A45A0008AC5A0008B15A0008A85A0008A95A00081C480008C9
:201C00002448000800000410445B000820480008B45A0008B05A0008B95A00080149086828
:201C2000704700BF244800080120704710B5084C2070084C2170084C2270084C2360084C43
:201C40002360084C02982060074C0398206010BDB95A0008B05A0008B25A0008A45A000811
:201C600080890008AC5A00081848000800B583B00021019102912F490022D24313460CC1DA
:201C80002D4B00210328197005D102AB6A4601A9012000F037F8284A00991078002805D04A
:201CA000264B01981860029A01F0FCFE03B000BD00B583B0204A0023019302931370022860
:201CC00002D11F490B6011E003280FD102AB6A4601A9022000F016F817490878002805D05E
:201CE000164A01981060029901F0F0FE03B000BD022804D0032804D11249086801E010498E
:201D00000868704730B5012808D0022811D10A4A012010700B480A460B4908E0064D06205D
:201D200028700448094C0460064C0C6008211060196030BD28480008AA5A000880890008B4
:201D4000009000080020031010000000AA55AA5530B51D4C00252078022811D11B480268C6
:201D6000002A06D01A4B19681A4B1868FFF7DAFE1BE019490878012804D11848057001E039
:201D8000032809D1164A25701570164A1178164A1078FEF7C1FF08E0124A1178124A10788D
:201DA000FEF7BAFF0E4A2570157030BD00B50F4A002010600A4A10700D4A11780A4A1078E8
:201DC000FEF7AAFF00BD00BFAA5A000820480008B45A00081C480008A85A0008A95A0008D6
:201DE000B85A0008B05A0008B95A000880890008B25A000800B50E4A012303210220FFF70A
:201E0000DBF8002001F0A6FA03F063F900BD00B503210220FFF72AF9002001F0C7FA00BD8F
:201E200000B5C82001F0EBFA03F053F900BD00BFA086010000B502F071FF03F04AF90948AF
:201E400002F09FF90021084602F0A8F800BD00B50221002000F098FE0121002002F09EF8F2
:201E600000BD00BF340B011000B584B0417901AA1170811D029101680079009110726946F2
:201E8000022002F0AAF804B000BD0020704700B502F074F802F07BF802F068F800BD0000BD
:201EA00000B5FFF7E2FA2649012008700220FFF7A4FB244A002304210846FFF77DF8224902
:201EC0000878224900014018007B312801D100F02CFB00BD00B51C4A1C49107800014018E3
:201EE000174AC07B117881420CD2FFF7BEFA1448144A017801310170002304210846FFF70C
:201F00005BF803E008210420FEF706FF00BD1048704730B5002305E0D41A0419CD5C013C1A
:201F2000257001339342F7D330BD10B5002302E0C45CCC540133013AFAD210BD70477047CC
:201F4000BA5A0008404B4C009A5A000890080110FF0F0000FBB583B0039055481746002645
:201F60000670544A925D012A04D0032A21D0072A4DD002E0039803281ED30136062EF0D32C
:201F80004D4807604D48059901604D4802784D48D20014588218002C44D0927900940192C3
:201FA000FB1C082207210420FFF740FE0620032149E00398032801D913212DE0421E424822
:201FC0005208002502700498029542781402827814433C4BEA009A1893889C4213D1D27971
:201FE000012A09D100F06DFB002805D13321029102990029C1D00FE031482D4A0570157869
:2020000001351570F4E701350E2DE2D3F0E728480278002AB1D13121059B3A462220FFF7ED
:202020008DFA1BE09288D1200002824202D1FFF7E7FA03E0254CA24203D101201E490A689D
:20204000D07004200721FEF767FE0120FFF7D5FA1F4A002304210846FEF7AEFF03B0FBBDA8
:2020600030B5154962220868174D0270144A15480C681378DB00C3189B881B0A637013783D
:202080000C68DB00C3189B88A3701278D20082180A48947909680368287840000019013085
:2020A0001880908801F008FA012030BD10207047BC5A0008900A01103048000834480008BB
:2020C000BD5A000828090110BE5A000821D00000A8610000FDB582B00290C1480C46002193
:2020E00001700091BF4EC04FC049009A895C062900D381E0012900D283E003D003292AD37C
:202100003CD07EE0029804287BD213216BE0FFF777FA012801D1312165E0A17800220D0280
:20212000E1780D4311468800431ADB009B191B899D4201D1397002E001310329F3D3C9B2AC
:20214000032900D1312211464BE000F0BAFA002857D1332147E000213B789A00D31ADB0008
:202160009B19CA186378127B934202D001310329F2D3C9B2032944D1122134E03B789A0047
:20218000D31ADB009B195B890298984201D0132127E0002125E0397800228B00591AC9009F
:2021A000891901920989FF200002814218D39048814215D88F48211D0422FFF7AAFE2146C1
:2021C0008D4808310422FFF7A4FE8B4B1968894B8A4A186800F0D9FC002801D13121019111
:2021E000019900290DD0049B039A3120FFF7A6F97B480121017025E00729A6D387D0082991
:20220000C9D000980130C0B20090082800D26BE77B49029A0A807B490C607B49039A0A6021
:202220007A490498086039788800411AC900895988470120FFF7E1F9754A00230421084683
:20224000FEF7BAFE02B0FDBD00B5674A10788100081A6449C00040184068804700BD624A37
:2022600010788100081A5F49C0004018007D704700B582B05F490868FFF7D6FC002817D168
:20228000644B012018700320FFF732FD072101300AD000230193009308220420FFF7C6FC1B
:2022A0000320FFF705FD06E00420FEF735FD02E059490120087002B000BD30B582B0554D8D
:2022C00000242878012836D324D0032814D332D14D4B1968444B18788200101A414AC000D0
:2022E00080180F300522FFF720FE484B1868052101802C7001241EE0019400942346082297
:2023000007210420FFF792FC0320FFF7D1FC0120287010E0384908220868019035480094A1
:20232000072103680420FFF781FC02210620FEF7F3FC03202870204602B030BD00B50121AF
:202340000520FEF7E9FC354A01201070344A00201060344A072110700420FEF7DDFC00BD7B
:2023600070B582B02D4D00242878012800D291E019D0032868D37ED0042800D08AE0224BEC
:202380001968194B18788200101A164AC00080180F300522FFF7C9FD1C4B186807210180B2
:2023A0002C70012476E0FFF7B2FD1E490A781C49104E0B68316853430F4EC9180238336800
:2023C000834202D91B1A013202E0184623462246134E3060084E3360124E3270094E23E0AE
:2023E000BF5A000898090110C15A0008980A011001FF0000384800083C480008BB5A000803
:2024000090580008404800084448000848480008A8610000C35A0008C05A0008C45A00089A
:202420004C480008C25A0008019000913068831C082207210420FFF7F9FB03210620FEF7E4
:202440006BFC0220287025E048490868484900900868831C08220721042000F05EFF02213F
:202460000520FEF759FC434A01201168002900D1032028700EE0404900940868431D08220C
:202480000721042000F049FF03210520FEF744FC04202870204602B070BD00B582B0374AD1
:2024A0001068013017D0364B012018700320FFF71FFC0721013003D00420FEF72DFC11E0CF
:2024C00000230193009308220420FFF7AFFB0320FFF7CCFB06E02A4A02200721107004209C
:2024E000FEF71AFC02B000BD00B5234B1968254B18788200101A244AC00080180F300522E6
:20250000FFF713FD214B062118681D4B01801878012803D0022805D1012000E00220164AAA
:2025200011684871012000BD704710B5154A10788100081A1449C00040180089FF2109025C
:20254000884212D112480478012C0ED10320FFF7CFFB013000D002240E4A002014700C4A90
:20256000072110700420FEF7D7FB10BD4C480008404800083C480008444800084006041055
:20258000C55A0008C15A00089809011048480008C05A0008C35A0008F0B51E460D46497843
:2025A00014464A06520E00234749C95C012925D305D0032911D316D00A2932D01EE00228EF
:2025C0001CD21321334622462720FEF7B7FF3F49002008703E49087072E0012A0ED0022A60
:2025E0000CD01221EEE70021012A02D1022802D102E0052800D013210029E3D10133052B87
:20260000D2D3344F012A2DD131490878002810D1FEF760FD38600028FAD02C49012008707C
:2026200009E0022AEAD1294F39780029E6D12421C8E700203860687801283DD167202070E7
:20264000012060703846A11C0322FFF76EFC0520308008210320FEF75FFB05210420FEF71A
:202660005BFB2DE03846FEF715FB00214A19435C9278934219D101310329F7D314490120E2
:2026800008701249002008706878022814D16720207002206070308008210320FEF73CFBAF
:2026A00005210420FEF738FB0AE03346224635212720FEF743FF03E006210420FEF72CFBBF
:2026C000F0BD034908787047A00A0110C75A0008C65A0008504800080349002008720349EC
:2026E00008707047704700BFD05A0008C65A0008F4B582B01E460D460021884B5B5C012B72
:2027000057D00A2B04D362D00C2B73D300D185E001310729F1D3821E814C8248214602805B
:2027200092B2A81CFFF701FC7F490C607F49029808607F4806607F480378687898427FD127
:202740007D4A012010707D4A14607D4CFFF766FA7C4A216840181060724A11887A4A7B4BC1
:2027600011601868401818606368984203D10120C007084310600120FEF73FFF744A002347
:2027800004210846FEF718FC6F4908686B4901900822086800906B48072103680420FFF7C6
:2027A00045FA04210620FEF7B7FA6A490220087059E0634A00249368DB0705D4022800D2E0
:2027C0001324002CA4D034E00328F9D3F9E75C4C0023277AFF070AD5564A17786A78013F95
:2027E000BA4205D0594A17686268974200D124231C46E6E74F4A002314786A78013CA242B1
:202800000AD0524A4E4C17683F186268023F974202D97123002222721C46D2E7454A6C783B
:2028200013789C4200D173E7013B9C4200D16FE773243346029A21463620FEF77FFE12E0F6
:202840004449032008703B49581E08700120FEF7D4FE3F4A002304210846FEF7ADFB072112
:202860000420FEF759FA02B0F4BD30B582B0394D00242878012849D338D0032811D345D1B6
:202880002B4A02211068294A01801068762101701068284A1178417001312C70117001241C
:2028A00034E02849086825490860FFF7B7F92A4A1168401A24490860FFF7B0F92649086015
:2028C000194803681F482049036008681B49019008220868009007210420FFF7A7F9032164
:2028E0000620FEF719FA012028700FE01649082208680090134807210368042000F00DFD6D
:2029000002210520FEF708FA03202870204602B030BD0B490020087272207047A80A0110BE
:2029200074480008925800086C4800087048000868480008C85A0008C95A000860480008A8
:20294000D05A0008644800085C48000854480008A8610000CB5A000858480008F0B581B08D
:2029600000243949095D032910D00A2915D1374E00213578002D05D0354F3D68354F7E683E
:20298000B54200D02421002903D106E0012804D013213720FEF7D2FD20E00134032CE0D3E5
:2029A0002D4802602D4829490360002008702C4901200870FEF721FE2A4A00230421084632
:2029C000FEF7FAFA00200090274B08220721042000F0A3FC03210520FEF79EF901B0F0BDB4
:2029E00030B582B01E4D00242878012815D0022821D11948016877220A70184A116803228A
:202A00000A80194902684B785370006809788170104804722C7001240DE0019400942346F2
:202A2000082207210420FFF701F905210620FEF773F902202870204602B030BD0549002056
:202A400008721020704700BFB00A0110C95A000854480008D05A0008785800087C580008D6
:202A6000CC5A0008A8610000CE5A0008F9B500900C46174600253E49495D06293DD2012948
:202A80000AD0032913D0052929D03BE0FFF719FE002837D133212AE0009805280AD331E0BD
:202AA0006178002919D1A178442916D12AE000980B2827D013211AE02E4EE11C30460422AE
:202AC000FFF727FAE11D301D0422FFF722FA2A4A03CE00F05AF8002814D1312107E0254822
:202AE00000218268D20700D5222100290AD0019B20783A46FEF722FD39E00729C6D3CFD08E
:202B00000829D9D00135062DB5D3FFF700FA194A91680322914301221143164A9160174A7C
:202B200001211170164A00211160164A0446116001210520FEF7F0F8742139702021797059
:202B40000021CA190220451AED00083D26462E41967001310229F4D3019A0421118008213F
:202B60000320FEF7D9F805210420FEF7D5F8F9BDB40A0110D05A0008BB5A0008C85A000862
:202B80005448000858480008704700B5FEF7AFFF00BD0000F4B581B0BB4A1578BB4A0E4658
:202BA000BB4C1078A84225D01F46691CC9B2032002F088FCB44A631C117061784C1EE4077D
:202BC000E40F1C702B03E818B24B019AC3181360B14C6B00079A1B5B33808B01C818AF4BCA
:202BE0004000C0181060AE48490040183860AD48405D1BE0AC48017801290FD10021017088
:202C0000019AAA481060AA4A10883080079AA9481060A948A94A1860107807E000203080DE
:202C200007999E4808609E481860012001B0F4BDF0B583B0002000F021FC041C00D168E186
:202C40009F4E036831688B4202D071688B42F1D1307B022805D3A079717B8842EAD1012024
:202C600000E00020974F38706579082DE2D301198A79F02111403029DCD801B47068924E05
:202C8000C01A00D0012033780290012B01BC00D9DBE00B1C49D10291082DCBD811070D0FCF
:202CA0000095C7D00722111A8D42C3DC774E01990029357809D10019C0793E2805D17A4AC5
:202CC00001210291117079480AE080490878002802D0184600F07FFA290368186D4940184F
:202CE0003A78A11D51184A1C0021535C4354009B01319942F9D302981A4600280BD166490D
:202D0000680042526748019A4255681CC1B2032002F0D8FB03E06648684E019902803170F3
:202D200000210120FEF78CFA84E7019A002A81D0102937D1002000F04EFA387801198A79EF
:202D40001207CB79120D06311A430823181A824200D26FE75E48824204D93221002000F070
:202D6000DAF867E75B4B002018705B480260474A107802038018474A821858488B1C002197
:202D8000026003E0585C50540131C9B238780624201A8142F6DB524A30211060002000F0D4
:202DA000BAF847E7202900D044E7484A1178022900D03FE7474A117801310907090F001926
:202DC000117082791207120F91423AD1444A434CC31D116820680D18002006E0195C295444
:202DE0001168013111600130C0B23B4C2668B14210D239780724611A8842EFDB3948426814
:202E00003948002301780320FEF7D6F83749042008700FE7002000F0DEF91C4E1E4A236859
:202E20003178480083521F48012242540131C9B2032002F047FB317000210120FEF700FAD6
:202E4000F8E6002000F0C7F9F4E6302900D0F1E60198002800D1EDE6032B00D0EAE61007A0
:202E6000000F07D12249088004203070002000F001F9DFE6022848D01D4AF521FF3110885E
:202E8000884242D236E000BF4D5B0008DD5A00084D5B00080C090008A058000808080008AB
:202EA00098580008DE5A0008F25A00080408000894580008000800089C580008DC5A000834
:202EC000F4090110E55A0008E45A0008E15A0008FF0F0000E25A000880580008E85A000898
:202EE000EC5A0008E0090110F0090110E35A0008A858000801301080C4484268C44800238D
:202F000041780320FEF758F894E6002000F06FF990E603B0F0BD10B584B001AA10700C4652
:202F200008215170BB4A91680091694600F094F9B94A6846811D107842180C540023537075
:202F400093700330C0B201E00B5401300828FBD3302C0CD1B14901200870B1480268AC4837
:202F600001780320FEF728F8AE49032008706846FEF77AFF04B010BDF0B584B000263446F8
:202F800030463546A84AA94F11784B00FB181F88002F06D01D808E018B19A54E3C465B0023
:202FA0009E190139C907C90F11700130C0B2002C07D10228E6D39F480488002C58D0058021
:202FC0009D4E01AA1570934A694690680090284600F042F9904B07221978501A844218DC70
:202FE00001AA0820507088188470C21C294602E0705C50540131E0B28142F9D319780723FD
:20300000591AC9B201E0155401308842FBD301201EE068460630220A10231A43425408183A
:203020004470821C01AB08205870284603E0335C13540130C0B206277B1A9842F7DB7F4982
:203040000E607F490B807F490D707F4902200C807E4908706846FEF707FF7D4901200870AD
:203060006A4802686A482B4641780320FDF7A4FF04B0F0BDF0B586B0744D012428780428B0
:203080005AD103AA00201070624A02A990680290002000F0E1F86B49087801300007000F73
:2030A00008705D49664F654E0B7802A95918202210438871CA1D398830680E180196002040
:2030C00007E0019E0131365C398089B216540130C0B20726F61AB04205DA01B45A480088B8
:2030E000814201BCEDD303AF08237B70F6B202E0002313540130B042FAD3534A10888142CC
:2031000002D300240520287002A8FEF7ADFE0020FEF7BBFE002801D0002C0BD14C4901202A
:2031200008703A4802683A48002341780320FDF743FF01E0012CAED006B0F0BD00B5374851
:203140000178012901D10221017040490878012805D0022810D004280AD0052819D1002018
:2031600000F045F8012200211046FEF779F810E00020FFF77FFF0CE0032008703449022078
:203180000870224842682248002341780320FDF713FF00BD00B5002000F006F800BD00B542
:2031A000002000F009F800BD00B51E4A1178002901D000F010F800BD10B5254904460878EF
:2031C000002807D0204600F012F8214600220120FEF746F810BD00B5104A00201070114ADC
:2031E00010700B4A03201178FDF740FF00BD00B5184A00201080154A1070154A1070044A8B
:2032000003205178FDF732FF00BD00BFE8090110F0090110F4090110E55A0008E15A00087D
:20322000E0090110E35A00084F5B000898580008080800089C58000800080008845800089D
:20324000AC580008F15A0008AA580008E45A0008F05A0008A85800080548027B022A03D399
:20326000407B8871012000E00020024908707047F4090110E55A000800B5FEF7DBFD00BD6B
:2032800000B5FEF7E4FD00BD2A49012008702A4908707047F0B5284D2878012804D0022857
:2032A0001ED00120287026E024480468402C03D9403C0460402401E002202870204E1D488F
:2032C000204F328803783868214600F0F1F8194F30801C490020387008680019086007E04D
:2032E000194A002028701178184A1078FDF714FD2878002803D002210520FDF70DFDF0BDAD
:2033000000B5104A10680E4A11880F4A018011780E4A1078FDF700FD00BD10B50B4C207098
:20332000094C21700A4C2270064C2360034C0298206010BDF85A0008F45A00088C58000818
:20334000F65A000888580008F95A0008F55A0008FA5A0008002828D172B60E4A01201060ED
:20336000022010600C4A0121C9071068084310600A4A0B481060084A102110680843106073
:20338000084A0121C907106808431060014A0320106009E040C0264010C0264008C0264025
:2033A0005019000000C0264062B67047002824D172B60D4B01201860022018600B4B002069
:2033C000186058600A4B0B491860586840084000586058681022904358605868084058605F
:2033E000014B0320186007E040C0264004C026400CC02640FFFEFFFF62B60020704700282B
:203400000DD072B604490120086002200860012048600320086001E040C0264062B67047DD
:20342000F0B581B01E4F1F4C3A7813011B190C689D1D042601B42088288002340235013EDB
:2034400001BCF7D1047900681C711860087958710132D2B2032A00D332463A700521032091
:20346000FDF75AFC01B0F0BD00B50F4A10780130107004210320FDF74FFC00BD0B4A084B71
:2034800011781878814209D0064B0801C0180131C9B2032900D30021117000E00020704740
:2034A000005B0008045B0008345B0008D15B000800B500F003F800BD7047000010B50A4C48
:2034C000012B00D0144622460AE00478130A63401402A2B2DBB2054C5B001B5B5A40013024
:2034E0000139F2D2104610BDFFFF000040060110F0B583B00023029300286DD0002A6BD0FC
:2035000001238B4014680193002C01D1436000E083603C4C137A041B3B4DE40924016519FC
:20352000DE06F60E1F27042908D2CBB2DB002C689F40BC439E4026432E6008E00B1FDBB218
:20354000DB006C689F40BC439E4026436E60019CE643846C53693440DB07DB0F8B402343E6
:203560008364C46C93693440DB07DB0F8B402343C364D36900934B001C4610340327C56C85
:20358000A740BD43009FBF07BF0FA7402F43C764546800948C000F27456CA740BD43009F44
:2035A0003F073F0FA7402F434764D7680325046C9D40AC43BD07AD0F9D40254305644369F6
:2035C000019B43614369836912693340D207D20F8A401A43826101E00C490291029803B04B
:2035E000F0BD10B500242101081B0949800040180246017900680832FFF77AFF0134022C90
:15360000F1D310BD000031400000304001005A00080C011000C3
:2036180000007047FEE7FEE704207146084202D0EFF3098001E0EFF3088000B5004FB84761
:203638001F360110FEE7FEE7FEE7FEE7FEE7FEE7FEE7FEE7FEE7FEE7FEE7FEE7FEE7FEE786
:20365800FEE7FEE7FEE7FEE710B564488208D2B2002004E0624C830001301C595C5061490E
:203678009042F7D3604A1160402210684422086410685E4A48641068000A000240210843D3
:2036980010605B491068084010605A4A012010600220106010BD00B5574B00201860586093
:2036B800564B01211860564B0904186888431860544B186888431860534B18688843186083
:2036D80018680121090588431860186801218904884318604D4B002018604D48302100F067
:2036F8002FF84B48322100F02BF84A4B186801231843484B01211860414B4904186808432D
:203718001860404B1868084318603F4B0121090418680843186018680121090508431860DC
:20373800374B01210904186808431860354B18680843186008200222052100F01BF800BD88
:203758004A09012A09D30ED0022A12D1403901228A40816D114381650BE001228A40016D36
:203778001143016505E0203901228A40416D11434165704730B5284B8000C318186807258E
:20379800A8434C07640F2043186018680124E407204318608807C00E9207130EFF2585401A
:2037B8008340002902DB8A08104C04E00A07120F083A9208194C920012191468AC431C435C
:2037D8001460002907DBCA06D20E154B0949012090401860086030BD704700BF800000003C
:2037F800000001100088000808ED00E000E400E0FF00FFFF00E100E050002140580021404F
:203818000013204080132040000024400C00214000002140C8002140008020401CED00E006
:2038380080E200E030B5034A034801241060A407024D05E0405B0008880A011000040040B3
:2038580072B6032080020019ED30FF300F210160084A0020A050084A13200002A050002094
:2038780001221203A05005482860286804482860286807E0180C00003C1000000F00FF8357
:203898000000FF8362B630BD05490020C0430860486004490020086003490448086070477C
:2038B80000182640081026400CED00E00400FA0510B572B60F4AF02110680F4A0840002187
:2038D800C94311600D4A0123FF33002418C20C4A090D11600B4A022111600B4A7721116084
:2038F8000A4A012114600A4AC9071460014A084310600FE080033940A0033940C4033940E1
:20391800CC033940B0033940D4033940F80339408803394062B610BD10B50C4672B6084ADD
:203938000121C907106808431060064A1460064A00201060054A102110680843106007E00C
:2039580080033940A003394088033940C003394062B610BD72B6074A1168074A1068000A4D
:20397800000210600846034A0121C9070843106004E000BF80033940C803394062B67047C3
:2039980010B572B601490C6802E000BF8803394062B6204610BD72B6164A174910684000D4
:2039B800400808401060154A0020C0431060144A00201060134A1449106808400121FF3143
:2039D800084310605068000A000250600F4AC32189001068084310600D4A1068000A0002CC
:2039F80010600C4A322010600B4A106840084000106013E080033940FFFFF8BFA0033940A2
:203A180088033940C4033940FF00FFFFCC033940B0033940D4033940F803394062B6704746
:203A3800062801D91F2001E00849085C704710B5074A117B884224D1064A074C1178002924
:203A58000CD10122032304210BE000BFBC0A0110C80A0110505B00087C5B0008FE22FC23CE
:203A7800FB216270A370E17072B6204600F03AFA62B6E088FFF7D4FF0021002803D1764905
:203A980001E0FF200021754A118010BD30B5744D02242C70734D01242C70734C734BE26028
:203AB800A06003C32161204600F036FAE088FFF7B7FF30BD10B56A4B02226B4C1A70694B8C
:203AD80003221A70A060E160204600F0E5F9E088FFF7A6FF10BD00B500F007F86449087809
:203AF800012801D100F02BF800BD00B5614B5D4A986900281BD11968002907D01078012894
:203B180004D15A69186900F064F817E01078032806D1D869196A814202D900F06DF80DE003
:203B38004F49002010700870FEF706F906E0002010704B4901200870FEF72CF900BD00B58A
:203B58004B4A4D481178012910D1002111704268002A05D0494B0068196800F014F805E0E6
:203B780040490A703E490A70FEF7E6F800BD30B53B4D02242C703B4D404B2C70044612C39C
:203B980000F001F830BDF0B5144600230125ED02AA4204D92C469E00375877500133A608EF
:203BB800B342F8D3AA4206D29B0002E0C55CCD5401339342FAD33148111BB30081604168F2
:203BD800C9184160016809190160294801210170F0BD30B5274C0D4600F006F96169202307
:203BF800203161612169203121610021202D00D3E91A2160A06130BD10B5044600F051F842
:203C180001210907611A1F221204914208D21C4A0121C9036118914205D20121C90301E095
:203C3800012149030A19174905C110BD10B503460A18002000290BD0042909D9124CA34242
:203C580006D3124B9A4203D8114A914200D8012010BD034908787047A5A50000785B0008C3
:203C7800FC5A0008FB5A00087C5B0008645B00087A5B0008545B00085C5B0008585B0008BD
:203C980000001F106C5B000800000410FFFF2010FFFF1C006749086801210843654908600F
:203CB800704700B500F009F8011C04D0624A0121904200D10421084600BD70B500265F4A09
:203CD80035465F4B1146044678C15E48012100F001F870BD10B581B0036804465A48002B77
:203CF80011D55A4BE2601A686B46009219800099A160E169002903D45049086800F00BF8A1
:203D180051498842F5D0524A116801221143504A116001B010BD010F0A2901D1002062E0D6
:203D38004C4A2921490490421ED24B4A90420FD24A4A904257D04A4A904252D0494A9042BA
:203D580033D0494A904201D1481C4CE047484AE0474A90422FD0474A9042F7D829D03E4AB3
:203D7800904224D9C81C3EE0434A90420BD2434A904227D823D0424A90421ED0354A904230
:203D9800E4D1881D2FE03F4A904227D03E4A904221D03E4A90421BD03D4A904215D0364A02
:203DB8009042D3D108460A301DE008461BE0881C19E0081D17E0481D15E0C81D13E008466E
:203DD800083010E0084609300DE008460B300AE008460C3007E008460D3004E008460E3050
:203DF80001E005200005704700B5114600F011F81E4988420BD0011C09D00F49884201D1EE
:203E1800042104E01D4A0121904200D10321084600BD10B5094A00231E4C53600523938093
:203E38001460906000230748D160D3710121FFF751FF10BD00F4244002005200945B000847
:203E5800000100140000224002005000C40A011008002440910000F0040000F00F00520060
:203E7800090000A0010000F0030000F0FFFF00000A0000F0060000F0A60000F0A40000F085
:203E9800920000F0BB0000F0B20000F0AA0000F0A80000F00001010610B50E4A04460E4943
:203EB8001068884201D0052011E0A068C20401D002200CE0E168002908D0084A09181160E6
:203ED800074A1060FFF798FE002800D10020E08010BD00BFA45B00083C3CA55A745B000823
:203EF800705B000810B504464078012805D1A078032802D1E078042801D0062005E0FFF7A5
:203F1800C9FE0349034808600020E08010BD00BFA45B00083C3CA55A10B50C4A04460C497F
:203F38001068884201D005200DE0A068420701D0022008E0E168002904D02269FFF749FE0A
:203F5800002800D10020E08010BD00BFA45B00083C3CA55A00B58D4A10684168006800F0C1
:203F78006DF900BD00B5894B186808224168006800F07FF900BD00B584490868006800F053
:203F980089F900BD70B5814A1068002460C8012904D30BD002290ED0012410E0287900F08B
:203FB80046FA3146284600F082F908E03146284600F087F903E03146284600F06FF9204696
:203FD80070BDF0B58DB005460E46002400F001FB002804D10621052000F017F90124002E6F
:203FF80005D10621012000F010F90124BAE0002C00D0B7E031790991B1680691317B376801
:204018000491002F05D4624862493840884205D809E06149B8008008884204D901240B20AD
:20403800062100F0F2F80498FF284ED10F20062100F0EBF8012495E0287E012804D1002CF2
:2040580002D10226344674E02046304371D102AA0499D07800F088F900F0D3F8099B0BAA4E
:204078000A9713700698243A0C90D6789279099203AA57780024002804D10621012000F0A3
:20409800C4F801240BA90878402808D8082810D92868C079002802D00A98400009D40621E9
:2040B800032000F0B2F80124FF21304600F05CF94AE0002CF8D100970AAB09983246019016
:2040D8000598294600F00FF93EE0002C4AD102A8C470047144718471C4710794089400F006
:2040F8008CF803A80130019001300090811E431CC21E284600F078F90646012819D003AA3E
:20411800107800F00BF903AA0590107800F014F905460598294600F079F8022801D001246C
:2041380008942868C079002886D1780084D50124079400F066F8002C00D13446012E03D12A
:204158000621022000F061F80898002803D00621084600F05AF80798002803D00B20062177
:2041780000F053F820460DB0F0BD70B5074C206060C8A86831460860284600F0A2F82846A7
:2041980000F0BDF80120207170BD07E0A85B0008FFFFFFBFFF070000FFFFFF1F72B67047D4
:2041B80062B6704770B585B01E466B46044600790D4611462A7E033300F0DBF804A9207955
:2041D800039608706946C87801A948730A98019009A80078087103A8FFF716F905B070BDFB
:2041F80030B5054600F0B4F8FF210446284600F0BBF82046FFF72CF930BD00B5FFF7C5FF83
:2042180000BD00B5FFF7CCFF00BD704710B5497A0124012903D30FD0032902D307D0002457
:204238000AE000F051F9022806D1044604E000F04BF9032800D10446204610BD70B50546F6
:204258000E460024FFF7D9FF284600F03DF901280BD1284600F0B5F90446707A022804D128
:2042780001207072284600F0A5F9FFF7CAFF204670BDF0B5174600240E46054600F02EFBF7
:20429800002805D03A463146284600F039FB04462046F0BD00B500F029FC00BD00B50022C5
:2042B8008A720A460968012300F039F900BD00B500220A76CA720A460968002300F02FF997
:2042D80000BD10B50C460021217600F073F90120607210BD0E49085C70470E49085C70473A
:2042F8000D49085C704710B582B005AC2478019404AC2478009400F085FC02B010BD10B5C7
:20431800044600F063FC204600F08EFB10BD00BFD80A0110E80A0110F00A0110694A014686
:2043380013682022D25C824204D9542041431868401800E000207047624A13682022D25CBB
:20435800824203D941015868401800E0002070475C4A13682422D25C002A03D0014618693A
:20437800405C00E010467047564B1A68126911547047FCB581B00192524A009001201768A1
:204398002122D65D002E2DD0002415E001B435196D10AB00D3181A780198824201BC0AD8A7
:2043B80006D39B788B4206D802D32C462E4603E06C1CA4B200E02E46BA68B442E6D3A40009
:2043D80014192278009B9A420CD1A2788A4209D10199002902D1E178012903D0029A617889
:2043F8001170002001B0FCBDF0B582B0354F01243D682426765D002E16D02035AE78002E9B
:2044180008D0864210D8ED78AD19A8420CDA801BC0B202E0ED78A84206D2089D0195079D0C
:20443800009500F022F80446204602B0F0BD70B5002113E0DB680A01D3181A7890420BD104
:204458005A689B689B1805E01E4E34682469FF25A55401329342F7D80131C9B2194A1368D3
:204478002322D25C8A42E5D870BDF0B5154C2668F6680001855D0D702568069FED682D18DD
:20449800A97B39702568059FED682D18697B39702568ED682D18297B19702168CB681B189C
:2044B80059689B685B18022007E025682D696D5CFF2D01D1117000200131994201D202280F
:2044D800F3D0F0BDA85B000800B55021095C406A00F0C3F80146C00703D4890603D40220FC
:2044F80002E0012000E0032000BD30B50D465021095C406A00F0B1F80446C0070DD4FFF7A8
:204518007CFE687A012804D10320A10600D402206872FFF776FE012000E0002030BDF9B569
:2045380084B0456A503005930678174600220C46B9880392002900D121882279013AD2B246
:204558000192A279013AD2B200926279531EDBB24A1E92B23146284600F09BF8227BFF2A91
:2045780005D0012003903146284600F095F9F988002900D1218A227A013AD2B20192A27A07
:20459800013AD2B20092627A531EDBB24A1E039892B202903146284600F097F8E37A059A9F
:2045B8003146284600F0D8F804983946FFF79DFF04B0F9BD00B55021095C406A00F0B0F85A
:2045D80000BD00B55021095C406A00F05CF800BD0000014908787047AC5B000849020818D5
:2045F80002657047002A01D1012202E0012A04D102224902081898231A50704749020818AE
:20461800F4300068C0B2704781B049020818F43000686A460090507801B0704749020818CA
:20463800006D704710B549020C189C22105900F060FBC0B220280CD39822105900F059FB98
:20465800C0B2FF21202802D21F21091AC9B2084602E03F21081AC0B210BD49020818806971
:20467800704749020918DC235858D83109688843D040C007C00F704749020818C4300068E7
:20469800C002C00E704749020818406C0006C00F704730B581B08B4D2C6805AD00942D78AB
:2046B8006C02D205D20D6D4622436A806B70009A04AD7F232D789A436B065B0E1A434902F0
:2046D80008180092C26101B030BD70B581B07E4E1F2424043568A543D406E40A25436E4659
:2046F8000095737005AE3678320106AE367833071B0F6E461A433270009B012207AED205D3
:2047180036789343F207120A1343490208180093C36001B070BD4902081880231A50704764
:2047380082B049020918886900906B4601201870009888610622FF3288690190C0B20128F1
:2047580001D0013AF8D2886900906A46032010700098886102B0704770B581B05B4E346812
:20477800032634432025AC43D507AD0E2C435A0001261643032212029443B207920D1443AE
:204798004902081800948461816989088900816101B070BD000081B049020818AC2319587D
:2047B8006B4600911A800099AC23195001B0704730B581B0464D2C6800940725AC432A4076
:2047D8001443702294435A07520E14432A0204AD2D7894436A07520D144349020818BC251D
:2047F8002C5001B030BD10B581B049020818842421586C4600912280A3700099842421505B
:2048180001B010BD81B049020818F82319586B4600911A700099F823195001B0704710B5C4
:2048380081B06C46A27023800122E270490208180099F024215001B010BD490208180121BF
:204858009140D02319507047F0B581B09206920E204E402515437F223468120694432A06C7
:2048780014436E46009406AFB3703F883780490208180099C026315001B0F0BD81B04902E6
:204898000818C82319586B4600911A700099C823195001B07047000010B581B00E4C4902C8
:2048B800081823686C46009362700099816401B010BD8A08920089071058C90EC840C0B2B5
:2048D800704700BFEC0B0110F00B0110F40B0110FC0B0110000C0110040C011030B50D4698
:2048F80000245021095C406AFFF798FE2A7E7D49012A00D17C49084000D00124204630BDB1
:20491800F6B59AB01B92436A0746503004930678744A0020099031461846FFF75FFE049813
:204938003146FFF77FFE079040200590079C3F2C6AD8788DBD6900222D1829200692C05D09
:20495800FFF7CBFC0830C0B260432C582D18600002D4E000440D06E0E000C0080124E40767
:2049780004438022069228460621FFF7A2FF830608D501239B071C430007000FFFF7AAFC35
:20499800039006E00107090F0391082901D90821039128460721FFF78CFF4006069A400EBF
:2049B8000243D2B20692039A9008C0B2930701D00130C0B2002309E008B40BA9099199001A
:2049D8004A19099B9268CA5008BC01338342F3D31B9802900AA80190039823460090069A65
:2049F8001A993846FFF7DEFB079A04983146FFF7F9FD04983146FFF715FE059D0790013D6C
:204A1800EDB20595002D91D104983146FFF706FE8822104005D004983146FFF7DFFD0120D4
:204A3800099009981AB0F6BDF0B589B005465035466A2F78039602973F22394604463046D0
:204A5800FFF769FE21462831487800903B200191035D31203946025D3046FFF7A9FEE06AF8
:204A7800618A0890A069002641180791218A636A421801983746049242882D78069305955B
:204A980018462946FFF787FE35461FE0069805992A46FFF7A7FDA8000899072240580028C4
:204AB80009D4B10000042843D2061043079A01368850F6B208E0F90052071043049A88505B
:204AD800501845600137FFB20135EDB201990878A842DBD80398628A02993346FFF783FE2A
:204AF80009B0F0BD1100080011000818F0B584B00646503604463178406AFFF78FFD029092
:204B1800C00428D5606A0090377820251BE000983946FFF779FD0190C000C11DE089A2694D
:204B38008018FFF7C6FE01221203039000983946FFF754FD019A00983946FFF763FE03983E
:204B5800FFF74EFBEDB200983946FFF757FD002801D9013DDBD20299480535D54620656AEA
:204B7800035D0195029301223678920231462846FFF734FD002524E02A4601983146FFF782
:204B980070FD00281BD02946204600F0A3F807460721FFF78EFEFFF7DBFBFF280FD03846D6
:204BB8000621FFF786FE0207120F039238460621FFF77FFE800602D50398FFF78BFB0135BB
:204BD800EDB20298A842D7D804B0F0BD70B581B0456A04465030E3890678227B314628464F
:204BF800FFF71DFE4434A0880090A378A27931462846FFF729FEE27831462846FFF73EFEB3
:204C180001B070BDF6B584B00BA905920F78416A06465030029101781D46019199681868F4
:204C38000391002802D44005C40804E0C000C0080124A40704434620805DB84204D8019983
:204C58000298FFF719FD074600973946304600F041F80646059A346010060124E4050443AA
:204C78002879FFF73DFB049A030717681B0B1C43FB79012B0AD12B685B0007D501235B05D8
:204C98001C43FB7A012B01D11B051C4374600836FFF720FB002313E0002427462979FA182D
:204CB800914202DD0399895C01E00CAA1178FA0091400C430137042FF0D310C60433DBB2A7
:204CD8008342E9D36A460BCA02461846FFF7B5FD04B0F6BD70B585690446463040780E4622
:204CF800FFF7FBFA08307043483421880818281870BD2021004202D0491E4008FCD108003B
:204D18007047000010B5304C2078002804D1042000F060F80120207010BD10B52A4C207831
:204D3800002804D0042000F0A7F80020207010BD254908787047F0B581B00E46224A0023D1
:204D58000093117801293BD1002839D11F4C204D204600F099F8217900278F420FD278000D
:204D7800815B207800F000F901372179FFB28F42F5D3207800F00EF900280FD10CE0207887
:204D980000F008F9002809D106E020782179013D00F000F9002801D1002DF6D1207900271B
:204DB800874209D2207800F0E6F87900013788532079FFB28742F5D3002D01D001210091B9
:204DD800009801B0F0BD00BFD25B000804480008FFFF000010B584B0A24AA34B0104891806
:204DF8001A68A24B00921A68A14B01921A68A14B02921A6803920A68520052080A60009A5E
:204E180003239B039A430123DB031A4303231B069A43994C81231B061A430092019A1023EF
:204E38001A4303231B069A430123DB071A4301922268FF231B029A430F231B021A4322600F
:204E58008E4C0123DB0722681A438D4B1A43920A92020D231A43029222608A4A800083187C
:204E78001868800A80020D2210431860019808620098086004B010BD7A4900044118086880
:204E98004000400808607047F0B584B00178754A090489180A6A03231B020092CA58012305
:204EB8005B020192CA5802920A6803920A68520052080A6042790924012A00D10424039AFC
:204ED8000F239A4322430123DB071A4303928279C3795400DB07DB0F1C436B46C4CB0C2329
:204EF8009A43A30744781B0F1A4303239B069A43A3071B0905791A430024012D00D9012433
:204F1800530832465B0023430126FF36047AB243E607F60D80783243461E1F208243F0065B
:204F3800C00E02430126FF36B743E607F60D37431F24A7430743029701920B6201980322B8
:204F5800120288500298012252026B1EC127BF008850C859FF2290431A06120E1043C85173
:204F78000398086004B0F0BD3E4A0004801809239B01C15070473B49000440180D2292015F
:204F980080587047374900044018406AC007C01701307047334A000480186123DB00C058CE
:204FB800C005C00D884201D0002000E0012070472C4900044018016849004908C1239B0081
:204FD8000160C158012212041143C1502E4AC1581140C15001680122D207114301607047DD
:204FF80010B5204A000480184B1E11D3026852005208C124A40002600159FF2291431A0611
:20501800120E1143015101680122D2071143016010BD1449000440183F2292018058C0077F
:20503800C00F70470F490004184A4118885801221043164A885070470A490004134A411869
:20505800885840084000885070470649000441183F2292018858012210433F22920188507F
:20507800704700BF00006040840C0110880C01108C0C0110900C011034100040000400409E
:205098000000FF03780C0040FFFFFEFFC80F0000704700B500F01FF900BD00B500F069F928
:2050B80000BD00B500F029F900BD00B500F049F900BD00B500F08CF900BD00B500F06AF904
:2050D80000BD00B500F0AEF900BD00B500F0C6F900BD000070B581B0C94E00246A46951CDF
:2050F800508029462046FFF726FE01280CD00134E4B229460020FFF71EFE012802D00A2C37
:20511800F5D304E00A2C02D2694648880612304601B070BD30B5BB4D00244620FFF7DAFF90
:20513800B749884207D0B8492C7208708006C00F6874012002E001202872204630BD30B578
:20515800B04D00244120FFF7C5FFAD49884207D0AE496C7208700006C00F2874012002E0A3
:2051780001206872204630BDB0B5A64D00244620FFF7B0FFA249884204D101202872287065
:20519800204617E0A24F2C72F8708006C00F68744120FFF79FFF9A49884204D10120687200
:2051B8002870204606E078716C720006C00F28742C700120B0BDF0B582B006460F460024F5
:2051D800019408028021314308436A46951C508029462046FFF7AFFD01280CD00134E4B240
:2051F80029460020FFF7A7FD012802D00A2CF5D308E00A2C06D23046FFF76CFFB84201D1DC
:2052180001210191019802B0F0BDF0B57D4E814C25462C356F1D00206871E871E07A032264
:205238001043E072E07804221043E070E0790C210843E071607A104360726079102108431A
:2052580060716078C0218843607041200021FFF7B2FF00283CD0E9794420FFF7ACFF002825
:2052780036D0E17A0420FFF7A6FF002830D0E1780220FFF7A0FF00282AD0E1790F20FFF71D
:205298009AFF002824D0617A1D20FFF794FF00281ED061790E20FFF78EFF002818D0617816
:2052B8000120FFF788FF002812D0002070703920397801552120E17A0155E0786076E07955
:2052D8006077607AE0776079E0766078E07501E001207070F0BD00B5FFF746FF002801D0DA
:2052F800FFF793FF00BD4749032802D90122002001E000220120CA72704730B5414D0028C6
:205318001CD1032903D90120E872002017E0414CE8720322E07A904311400843E072FFF7D1
:2053380007FD012808D1E17A0420FFF744FF002802D02120E17A0155002000E001202873EF
:2053580030BD10B5002812D1FFF7F2FC324C012805D10420FFF7BEFE2949884203D1607859
:205378008007800F04E060708007800F00E0002010BD704710B5274C0320E17CFFF71BFFE9
:20539800002803D02920E17C015502E01D490120487310BD10B51F4C0722E07C904304225F
:2053B80010432021884380210843E074FFF7C0FC01280CD1E17C0320FFF7FDFE002803D012
:2053D8002920E17C015502E00E490120487310BD10B5104C0722E07C90432421084380212D
:2053F8008843E074FFF7A4FC01281AD1E17C0320FFF7E1FE002811D02920E17C015510E082
:20541800FFFF0000D45B00081F5C0008215C00081C5C0008E85B0008085C00081D49012079
:20543800487310BD10B51C4C0722E07C904306221043A0218843E074FFF77AFC01280CD17A
:20545800E17C0320FFF7B7FE002803D02920E17C015502E00F490120487310BD10B50E4C10
:205478000722E07C10432021884380210843E074FFF75EFC01280CD1E17C0320FFF79BFE8B
:20549800002803D02920E17C015502E001490120487310BDD45B0008E85B000800B5011CD4
:2054B8000A2000F003F808BC1847000060B400230125021C04D10B4A002A10D060BC10477A
:2054D800914207D3891A5B194E08B242F8D252006D00F5E7012D02D052086D08F0E7181C67
:2054F80060BC70470000000060B50E1C00DC4942051C00DC4042FFF7D9FF002E00DA49423B
:20551800F60FED0FAE4200D0404260BC08BC184700000000040110010100000100000000D9
:040000051020E640A1
:00000001FF
